:1042700000010C01010602011E030A960401320529
:10428000050506006407010108000009015A0E0136
:10429000010F000112006413010114013C1501FA21
:1042A0001664FA17FFFF1D000720000724000227ED
:1042B00001012F013C30030332010335FFFF3603B8
:1042C000073CFFFF3DFFFF180002191E461A0002BF
:1042D0001B00022D32C82E0001FAFAFA180000194C
:1042E000FFFF1A00001B00002D32C82E0001FAFA51
:1042F000FA18000019FFFF1A00001B00002DFFFF35
:064300002EFFFFFAFAFA9D
:10004800900787E0FEA3E0FF7457BE0010D39F40DF
:100058000C90427012001EE493F599804C900014A5
:10006800E0D394044014900787E0FEA3E0FF904299
:100078007012001EE493F599802F900014E0D39439
:10008800034014900787E0FEA3E0FF90428512002A
:100098001EE493F5998012900787E0FEA3E0FF9095
:1000A800429A12001EE493F59990078712000E9069
:1000B8000787E0FEA3E0FF746C6F4E7003751300B2
:1000C80022900073E0B402087401900073F0D20E1D
:1000D80090013BE090002AF090013CE090002BF06A
:1000E80090013DE090002CF0A20AB3401690013B2D
:1000F800E0700C90013CE0700690013DE0600280E9
:1001080002C20A90013BE0B4300F90013CE0B447D2
:100118000890013DE0643B60028004D20B8002C27B
:100128000BE558B40102800302024B900058E0F539
:1001380066900063E0F568900064E0F569900075EA
:10014800E0F56A90007BE0900029F090007DE0F5F2
:100158006590007EE0F567900081E0F5649000828C
:10016800E0F563900091E0900041F0900092E090FB
:100178000042F0900093E0900043F0900094E090EB
:100188000044F0900095E0900045F0900096E090D3
:100198000046F0900097E0900047F0900098E090BB
:1001A8000048F090009AE0900033F090009BE090B7
:1001B8000034F090009CE0900035F090009DE090B5
:1001C8000036F090007AE0B4011790000A740FF03E
:1001D800A374FFF090000CE4F0A3F0740290007A8E
:1001E800F090007AE0B4035990000CE0FEA3E0FF21
:1001F80090000AE0FCA3E0FD12000374101243858E
:100208007408124377EF900026F0EF700674FF90A1
:100218000026F0740090007AF090000BE090002720
:10022800F090000AE0900028F0900026E090078AFD
:10023800F0900027E090078BF0900028E090078C62
:10024800F0803F900082E07006755801756300A247
:100258000AB3402E90013BE090002AF090013CE068
:1002680090002BF090013DE090002CF090002AE0E7
:10027800700C90002BE0700690002CE06002800269
:10028800C20AE5667003756602E568700375680260
:100298007E897FAFE5668E048F05FF1243678C3930
:1002A8008D3AE56975F0FAA4FFAEF0E5688E048F23
:1002B80005FF1243678C3D8D3E900050E0F560903D
:1002C800004DE0FE90006AE0B5061890004CE0FE94
:1002D800900069E0B5060C90004BE0FE90005AE0F3
:1002E8006E606F90006AE07006900069E0600674C6
:1002F8000090005AF090006AE0B402089000497437
:1003080001F08005900049E4F0900069E0B402082B
:1003180090004A7401F0800590004AE4F09000696A
:10032800E0600690004AE060028005756005800381
:10033800756006E559B55802D20E900069E0900044
:100348004CF090006AE090004DF090005AE0900068
:100358004BF0740090009FF074019000A0F07401BD
:100368009000A1F074009000A2F074019000A3F036
:1003780074009000A4F074019000A5F0740090003F
:10038800A6F074019000A7F074019000A8F0740022
:100398009000A9F074019000AAF074009000ABF0EE
:1003A80074019000ACF074019000ADF074019000FD
:1003B800AEF074019000AFF074009000B0F07401DA
:1003C8009000B1F074009000B2F074019000B3F0A6
:1003D8007400900363F07401900364F07401900357
:1003E80065F07400900366F07401900367F0740080
:1003F800900368F07401900369F074019003A3F00E
:1004080074019003A4F074019003A5F074009003A4
:10041800A6F074019003A7F074009003A8F074018B
:100428009003A9F074019003E3F074009003E4F0E2
:1004380074019003E5F074009003E6F074019003F2
:10044800E7F074009003E8F074019003E9F0740198
:10045800900423F07400900424F07400900425F0B4
:100468007400900426F07401900427F0740090043E
:1004780028F07401900429F07401900463F074006A
:10048800900464F07400900465F07401900466F0C0
:100498007400900467F07401900468F0740090048C
:1004A80069F074019004A3F074019004A4F074003E
:1004B8009004A5F074019004A6F074009004A7F0CD
:1004C80074019004A8F074009004A9F022E5B554D2
:1004D800F7F5B5E5B554FDF5B5C293C294C292C21D
:1004E80087C290756F00757000C207E5B554FBF5BB
:1004F800B5755106E55104F552900050E0F560904D
:100508000025E4F0C20990004EE4F0E5B554FEF58C
:10051800B5C28E758D00758B00754C0075260075FB
:100528002500D28E22750A00750900AE09AF0A743B
:1005380057BE00039F50030205EA90427012001E46
:10054800E49390004F12439D0FBF00010EE0FC9012
:10055800427012001EECFEE493FFEEC39F5026AEDD
:1005680009AF0A0FBF00010E90427012001EAE09BB
:10057800AF0AE493FC90427012001EE49390004F7F
:1005880012439DECF0AE09AF0A90427012001EE4CF
:100598009390004F12439DE0FC90427212001EECB3
:1005A800FCE493FDECD39D401990427212001EE4C6
:1005B80093FC90427012001EE49390004F12439DEA
:1005C800ECF0AE09AF0A74022FFF50010E8E098FAE
:1005D8000A780A740126F6500418E436F640030235
:1005E800053322750A00750900AE09AF0A7415BEF5
:1005F80000039F50030206B89042C712001EE493FE
:1006080090004F12439D0FBF00010EE0FC9042C7BF
:1006180012001EECFEE493FFEEC39F5026AE09AF16
:100628000A0FBF00010E9042C712001EAE09AF0AA2
:10063800E493FC9042C712001EE49390004F1243CB
:100648009DECF0AE09AF0A9042C712001EE49390E9
:10065800004F12439DE0FC9042C912001EECFCE4DE
:1006680093FDECD39D40199042C912001EE493FCFF
:100678009042C712001EE49390004F12439DECF085
:10068800AE09AF0A740F6F4E7006750A157509002A
:10069800AE09AF0A74022FFF50010E8E098F0A7837
:1006A8000A740126F6500418E436F640030205F1F0
:1006B80022750A00750900AE09AF0A7415BE000359
:1006C8009F50030207869042DC12001EE4939000BC
:1006D8004F12439D0FBF00010EE0FC9042DC120058
:1006E8001EECFEE493FFEEC39F5026AE09AF0A0F3F
:1006F800BF00010E9042DC12001EAE09AF0AE4935F
:10070800FC9042DC12001EE49390004F12439DECD3
:10071800F0AE09AF0A9042DC12001EE49390004F3D
:1007280012439DE0FC9042DE12001EECFCE493FDB7
:10073800ECD39D40199042DE12001EE493FC9042D7
:10074800DC12001EE49390004F12439DECF0AE09BA
:10075800AF0A740F6F4E7006750A15750900AE0959
:10076800AF0A74022FFF50010E8E098F0A780A749F
:100778000126F6500418E436F640030206BF227537
:100788000A00750900AE09AF0A7415BE00039F5030
:10079800030208549042F112001EE49390004F1295
:1007A800439D0FBF00010EE0FC9042F112001EECC9
:1007B800FEE493FFEEC39F5026AE09AF0A0FBF00B9
:1007C800010E9042F112001EAE09AF0AE493FC90AC
:1007D80042F112001EE49390004F12439DECF0AEDC
:1007E80009AF0A9042F112001EE49390004F1243A1
:1007F8009DE0FC9042F312001EECFCE493FDECD368
:100808009D40199042F312001EE493FC9042F112AD
:10081800001EE49390004F12439DECF0AE09AF0A1E
:10082800740F6F4E7006750A15750900AE09AF0A88
:1008380074022FFF50010E8E098F0A780A74012660
:10084800F6500418E436F6400302078D22054D22BF
:10085800054C22054EC2CF2290F800E4936406604E
:100868000280FE75840175A70075FF80900789E4F2
:10087800F075C91075A70F75A1C775A70075D900C0
:1008880075CEFF75A70F75F1FE75F2FF75F3377515
:10089800F47875A4BA75A5FF75A60775AE0075AF8F
:1008A800FF75D48175D5FF75D6FF75D7FFC296C27F
:1008B80095C2A0C297C2A2E5B554EFF5B5E5B55407
:1008C8007FF5B5E5B554F7F5B5E5B554FDF5B5755E
:1008D800A70075A20175A14775F80975BC0175BE19
:1008E8000475BD6C75BE0775BDA075BE0875BD01E4
:1008F80075BC0075BB1875BC2075BA0875E880759D
:10090800D11375A70F75E10575E20075C740759796
:1009180000759780740A1243577597C0E59754205D
:10092800700280F8758F0275A700D2AF75980075B0
:10093800A90C75A70F75AB4375ADFB75AC1E75A7F4
:1009480000758911758E00758C00758A00D2A9D240
:100958008C758D00758B00D2ABD28E75CD0075CCA1
:100968000075CA0075CB00D2ADC2CFD2CA7591044A
:100978007592007593CD75EF0675D94075CF0190C6
:100988000787E4F0A3F0751300751400C299D20A22
:10099800C2101204D574C8F518751700122ABE754E
:1009A800A70FE5FB90001AF0E5FA90001BF0E5F9B7
:1009B80090001CF075A70090F800E493F508122B3E
:1009C800F512312F90078AE0900026F090078BE00F
:1009D800900027F090078CE0900028F090078DE0B9
:1009E800900029F090078EE0F56690078FE0F56893
:1009F800900790E0F569900791E0F56A900792E01A
:100A0800F565900793E0F567900794E0F564900723
:100A180095E0F563900796E090002AF0900797E03C
:100A280090002BF0900798E090002CF0900799E048
:100A3800900041F090079AE0900042F090079BE008
:100A4800900043F090079CE0900044F090079DE0F0
:100A5800900045F090079EE0900046F090079FE0D8
:100A6800900047F09007A0E0900048F09007A1E0C0
:100A7800900033F09007A2E0900034F09007A3E0D4
:100A8800900035F09007A4E0900036F074009000D4
:100A980083F090013BE0700C90013CE070069001FF
:100AA8003DE060028004C20A8002D20A90F807E49E
:100AB80093900021F0900021E0440A900021F090EA
:100AC8000021E054FE900021F07406900012F074AA
:100AD80002900013F090F802E493900014F074036D
:100AE800900015F07403900016F07404900017F04D
:100AF8007405900018F0900014E0B4040674049093
:100B08000018F0900014E0B403067403900018F085
:100B18007405900019F090F804E49390001DF074A7
:100B28000090001EF090F805E49390001FF090F8F4
:100B380006E493900020F074FF900022F074419036
:100B48000126F07442900127F07436900128F07461
:100B580030900129F0742090012AF0744190012B03
:100B6800F0743790012CF0743690012DF0743190A8
:100B7800012EF0744590012FF07420900130F0742C
:100B880036900131F07453900132F0747090013353
:100B9800F07464900134F090007BE0D39401400637
:100BA800740090007BF0755801755901740390002A
:100BB8004CF01200C912052D900014E0B40405127F
:100BC80006B98011900014E0D3940440051205EB97
:100BD8008003120787122AEAE5B554FEF5B590009E
:100BE80025E4F0900787E4F0A3F07524007523004E
:100BF800754800752A007529007549007532007519
:100C08003100754A00755400755500755A007551C4
:100C18000675520175343C753300757200757100A4
:100C28007573CD755600755700754300754400758A
:100C38004500754600755B007547007542007541B3
:100C480000900006E4F0A3F0900008E4F0A3F0752B
:100C58005E00755F0090000E74FDF0A374E8F090DC
:100C68000023E4F07464900024F0C200D201C202B0
:100C7800D203754D00756D00E5B554DFF5B5C2A119
:100C8800E5B554BFF5B5C20FC291C20E7E017F0013
:100C9800900028E0124385900027E02FFF50010EB6
:100CA80090000AEEF0A3EFF0900026E0700674FFC3
:100CB800900026F090000AE0FEA3E0FFEFD394FF37
:100CC800EE940F400790000AE4F0A3F0740090003F
:100CD80072F0740090007AF07400900083F0740051
:100CE80090008EF074009000B5F0E56770037567AA
:100CF80004743A90074FF074FD900750F090045533
:100D0800E0900495F0D2B0D2B7D2A7D2A6D2B1D291
:100D1800A3C207A2B6B39204A2B3B39205D29CD2DF
:100D2800EC75CF01A298B34005C298123493E5132D
:100D38006006A299B3B340028005C299123A03E54E
:100D48001464016005E514B4040280D5E54DD3941C
:100D580005400CE55AC394C85002055A754D00E584
:100D680073C394F0501A787112003FAE71AF72EFEE
:100D7800D394E8EE9403400805737572007571000A
:100D8800C28E7E047F00E54C124385E58D75F00424
:100D9800A4FDACF0EF2DFDEE3CFCE58B75F0408436
:100DA800FF7E00ED2FFFEC3EFE8E258F26D28EA211
:100DB800B6300401B35003020F19A2B6300401B3D0
:100DC8005003020F19A2B640670554A210400575DA
:100DD800FFA0D210E5B54401F5B5900024E4F0E594
:100DE80054D3956640487C897DAFAE25AF26124125
:100DF8008F8E238F24E5482FFF50010E7401124374
:100E0800778E238F24852448755401C28E758D00F2
:100E1800758B00754C00D28E7403BE00039F50067C
:100E28009000257401F0E543B40603754300D2042D
:100E3800A2B6B35003020F19C20490006CE0601808
:100E4800123B44A200B34008E5B54408F5B5800656
:100E5800E5B554F7F5B58002C20090006FE0601860
:100E6800123C99A202B34008E5B54402F5B58006E4
:100E7800E5B554FDF5B58013A20FB34008E5B544B8
:100E880002F5B58006E5B554FDF5B5A207B34008EF
:100E9800E5B54440F5B58006E5B554BFF5B5900015
:100EA8005AE06004D20F8002C20F90004AE0B401F9
:100EB80008E5B54420F5B58006E5B554DFF5B590ED
:100EC8000049E0B40104D2A18002C2A1A209B34042
:100ED80004D2918002C291900018E0FE900014E0C4
:100EE800C39E4009900014E0D39408400974FB9015
:100EF8000023F01204D590001DE0601590001DE05D
:100F0800FE900017E06E600974FE900023F0120452
:100F1800D5C2CA7E017F00E54E124385E5CD2FFF7D
:100F280050010E8E278F28D2CAE565B4014890007B
:100F38000EE0FCA3E0FDEFC39DEE9C4039B208E54E
:100F48002A45296013A208B34008E5B54404F5B55D
:100F58008006E5B554FBF5B590000EE0FEA3E0FF72
:100F6800900010E0FCA3E0FDEF2DFDEE3CFC9000AE
:100F78000EECF0A3EDF0A2B3300501B3500302105C
:100F880067A2B3300501B35003021067A2B3500340
:100F98000210600555A210400575FFA0D210E5B5F6
:100FA8004401F5B5900024E4F0E555D39568500365
:100FB80002105E7CEA7D60AE27AF2812418F8E2931
:100FC8008F2AE56912438574FF8E048F05FF12434B
:100FD800678C298D2AE5492DFD50010C74018C067A
:100FE8008D071243778E298F2A852A49A209B34093
:100FF800157464124385900068E08E048F05FF1213
:1010080043678C298D2A75550190000EE0FEA3E0F8
:10101800FFAC27AD2812000390000EEEF0A3EFF00E
:10102800E567FF124367740AFF12436790007CE08C
:101038008C068D0712438574148E048F05FF1243A6
:1010480067900010ECF0A3EDF0C2CA75CD0075CC26
:1010580000754E00D2CAD205A2B3B34002C20590B1
:101068000025E0B40107E556C3940640030216873D
:10107800E56D902A9DF828287390005AE0C39402E1
:1010880040030211D5E551D3940150030211D5E56F
:101098005175F040A4FFAEF090031312001EE0C398
:1010A80095455018E55175F040A4FFAEF090031235
:1010B80012001EE0F52E752D000211D5E55175F0D0
:1010C80040A4FFAEF090031112001EE0C395454006
:1010D80003021171E55175F040A4FFAEF0900312C0
:1010E80012001EE55175F040A4FFAEF0E0FC90033D
:1010F8001012001EECFEE0FFEEC39FFEE5518E04C9
:1011080075F040A4FFAEF090031112001EE0F40445
:1011180025458C0088F0A4FFAEF0E5518F048E05BC
:1011280075F040A4FFAEF090031312001EE5517550
:10113800F040A4FFAEF0E0FA90031112001EEAFEA0
:10114800E0FFEEC39FFECDCCCD8E07124367E5517D
:1011580075F040A4FFAEF090031012001EE02DFDC4
:1011680050010C8C2D8D2E8064E55175F040A4FF44
:10117800AEF090031012001EE55175F040A4FFAECA
:10118800F0E0FC90030F12001EECFEE0FFEEC39FA0
:101198008545F0A4FFAEF0E5518F048E0575F0404B
:1011A800A4FFAEF090031112001EE0FECDCCCD8E50
:1011B80007124367E55175F040A4FFAEF090030FA6
:1011C80012001EE02DFD50010C8C2D8D2E756D0129
:1011D80002168790005AE0C39402400302138990D4
:1011E8000050E0D395515003021331E55175F0409A
:1011F800A4FFAEF090031912001EE0C395455018E5
:10120800E55175F040A4FFAEF090031812001EE0FF
:10121800F52C752B00021331E55175F040A4FFAE93
:10122800F090031712001EE0C3954540030212CD4B
:10123800E55175F040A4FFAEF090031812001EE5CA
:101248005175F040A4FFAEF0E0FC90031612001EAA
:10125800ECFEE0FFEEC39FFEE5518E0475F040A45E
:10126800FFAEF090031712001EE0F40425458C0031
:1012780088F0A4FFAEF0E5518F048E0575F040A408
:10128800FFAEF090031912001EE55175F040A4FF5F
:10129800AEF0E0FA90031712001EEAFEE0FFEEC37C
:1012A8009FFECDCCCD8E07124367E55175F040A463
:1012B800FFAEF090031612001EE02DFD50010C8CBD
:1012C8002B8D2C8064E55175F040A4FFAEF090039F
:1012D8001612001EE55175F040A4FFAEF0E0FC9038
:1012E800031512001EECFEE0FFEEC39F8545F0A437
:1012F800FFAEF0E5518F048E0575F040A4FFAEF007
:1013080090031712001EE0FECDCCCD8E0712436766
:10131800E55175F040A4FFAEF090031512001EE0F1
:101328002DFD50010C8C2B8D2CE551B40123E5606B
:10133800D39401401CE55604D395514014E545C3A8
:101348009405500D900360E0A829B80006952A403E
:10135800028003755102E551B56022900050E0D338
:1013680095514019E55175F040A4FFAEF09003186F
:1013780012001EE0A823B80006952440028002054A
:1013880060756D0202168790005AE0B4022AE55192
:1013980075F040A4FFAEF090031812001EE0F52C83
:1013A800752B00E55175F040A4FFAEF090030F12C5
:1013B800001EE0F52E752D0090005AE0B4030F9042
:1013C8000052E0F52C752B00752E00752D00756DFB
:1013D80003021687E55175F040A4FFAEF090032193
:1013E80012001EE0C3955A40030214B1900049E070
:1013F8007036E551D394014029AE23AF24AC2DAD0E
:101408002EEDD39FEC9E401AE55175F040A4FFAE37
:10141800F090031F12001EE0A829B80005D3952AF2
:101428005002800215518034E551D394024029AE10
:1014380023AF24AC2DAD2EEDD39FEC9E401AE55181
:1014480075F040A4FFAEF090031F12001EE0A8291B
:10145800B80005D3952A500280021551E551B552BE
:1014680037E551C395605030E55604D3955140286F
:10147800AE23AF24AC2BAD2CEFD39DEE9C4019E5E9
:101488005175F040A4FFAEF090032012001EE0A8B2
:1014980029B80006952A400280020551C290E551FC
:1014A80065526005C207755A00756D04021687E516
:1014B8005175F040A4FFAEF090031B12001EE0B47B
:1014C8000117E55175F040A4FFAEF090032112001A
:1014D8001EE0240AC3955A400302158775306475C7
:1014E8002F00A207B3500B900061E02405C3954577
:1014F8004003021587E55175F040A4FFAEF0900354
:101508001E12001EE0C395454064E55175F040A4E5
:10151800FFAEF090031D12001EE55175F040A4FFC8
:10152800AEF0E0FC90031C12001EECFEE0FFEEC3E0
:101538009F8545F0A4FFAEF0E5518F048E0575F048
:1015480040A4FFAEF090031E12001EE0FECDCCCDED
:101558008E07124367E55175F040A4FFAEF0900383
:101568001C12001EE02DFD50010C8C2F8D30AE2377
:10157800AF24AC2FAD30EFD39DEE9C4002D207755F
:101588006D05021687E551B4010990005AE0C3942D
:1015980002400302165B900359E0D39545500302BD
:1015A800165B900357E0C395455040900358E0FE02
:1015B800900356E0F4042EFE900357E0F40425450A
:1015C8008E0088F0A4FFAEF0900359E0FC9003571A
:1015D800E0F4042C8E048F05FF124367900356E055
:1015E8002DFD50010C8C2B8D2C802C900356E0FE89
:1015F800900355E0F4042E8545F0A4FFAEF0900367
:1016080057E08E048F05FF124367900355E02DFDC8
:1016180050010C8C2B8D2CE551C395605030E5564C
:1016280004D395514028AE23AF24AC2BAD2CEFD377
:101638009DEE9C4019E55175F040A4FFAEF0900373
:101648002012001EE0A829B80006952A400280034F
:10165800755102900049E0B40106E5516401600249
:101668008003755102E55165526005C207755A003D
:0F167800E55AD3940A400590004EE4F0756D00DA
:102A9D000210810211DB02138F0213DC0214B70244
:022AAD00158D85
:10168700900051E02402A823B80007D39524400214
:10169700C207900025E0B4010990005AE0C3940303
:1016A700400302181B900049E06003021764E551EC
:1016B700D39401403A90004EE07034E55175F04004
:1016C700A4FFAEF090031512001EE0A823B8001F78
:1016D700D39524401AE55175F040A4FFAEF090036E
:1016E7002012001EE0A829B80005D3952A500280D1
:1016F700021551E551D39401402FE55175F040A4EF
:10170700FFAEF090031312001EE0C39545501AE593
:101717005175F040A4FFAEF090031F12001EE0A821
:1017270029B80005D3952A500280021551E551D3F7
:1017370094014022E55604C39551501AE55175F0BE
:1017470040A4FFAEF090031F12001EE0A829B800C6
:1017570005D3952A500280021551021810E551D37E
:101767009402403A90004EE07034E55175F040A481
:10177700FFAEF090031512001EE0A823B8001FD398
:101787009524401AE55175F040A4FFAEF090032070
:1017970012001EE0A829B80005D3952A500280023E
:1017A7001551E551D39402402FE55175F040A4FF40
:1017B700AEF090031312001EE0C39545501AE55191
:1017C70075F040A4FFAEF090031F12001EE0A82999
:1017D700B80005D3952A500280021551E551D394DC
:1017E700024022E55604C39551501AE55175F04061
:1017F700A4FFAEF090031F12001EE0A829B8000551
:10180700D3952A500280021551E55165526005C2F1
:1018170007755A00900061E0D3954550099000552F
:10182700E0C395455002C20790005AE07003021AC0
:1018370080A2A5B34008A2A4B34003021A69AE353B
:10184700AF367441D39F749C9E4005783512003F94
:10185700AE35AF36EFB48806EEB413028003021A32
:1018670046A2A5500302190990005AE0B4010B9053
:101877000050E0D395604002056090005AE0B40242
:1018870054E55175F040A4FFAEF090032112001EFD
:10189700E0C3955A503F900050E0D395514021E561
:1018A7005604D395514019E55175F040A4FFAEF0A9
:1018B70090031512001EE0A823B8000695244002E5
:1018C70080020551900050E0F560E55165526005D2
:1018D700C207755A0090005AE0B40326900050E002
:1018E700D395514008E55604D3955150028002051F
:1018F70051900050E0F560E55165526005C20775EB
:101907005A00A2A45003021A4690005AE0B4016E8E
:10191700900049E07035E551D394014029E55175B0
:10192700F040A4FFAEF090031F12001EE0A829B8F4
:10193700000FD3952A400A1551755A0085516080CA
:101947000385516080037560018033E551D39402AC
:101957004029E55175F040A4FFAEF090031F120037
:101967001EE0A829B8000FD3952A400A1551755AC9
:101977000085516080038551608003756002900087
:101987005AE0D394015003021A3AE55175F040A486
:10199700FFAEF090032112001EE0C3955A400302E8
:1019A7001A3A900049E07041E551D394014034E57B
:1019B7005175F040A4FFAEF090031212001EE0A88C
:1019C70023B8001FD39524401AE55175F040A4FFB2
:1019D700AEF090031F12001EE0A829B80005D395AA
:1019E7002A500280021551803FE551D394024034BA
:1019F700E55175F040A4FFAEF090031212001EE00F
:101A0700A823B8001FD39524401AE55175F040A4C8
:101A1700FFAEF090031F12001EE0A829B80005D3FF
:101A2700952A500280021551E55165526005C2079B
:101A3700755A00E556B40704055E8003755E00E538
:101A470063B4010EAE35AF36EF64407005EE649CAB
:101A57006002800EA2A54003755801A2A440037539
:101A67005802A2A5B3B35006A2A4B3B3400280069E
:101A7700753600753500021B76A2A5B34008A2A4EF
:101A8700B34003021B62AE35AF367441D39F749CDB
:101A97009E4005783512003FAE35AF36EFB4880665
:101AA700EEB413028003021B62A2A540779000697F
:101AB700E0606290004AE0B4010790004AE4F080D9
:101AC7000690004A7401F090004AE07005756005C1
:101AD700800375600690004AE0B40108E5B544202C
:101AE700F5B58006E5B554DFF5B5E551B4061AE559
:101AF7005175F040A4FFAEF090031F12001EE0A83E
:101B070029B80005D3952A50028008755105C207E8
:101B1700755A008003756006E556B40704055E80B4
:101B270003755E00A2A4403390006AE06021900034
:101B370049E0B40107900049E4F080069000497439
:101B470001F0900049E0B40104D2A18002C2A1E5EE
:101B570056B40704055E8003755E00A2A5B3B350B3
:101B670006A2A4B3B340028006753600753500E5BA
:101B77005865596006900083E06003021CFEC29C12
:101B8700751400751300C2CAE558902AAFF82828C3
:101B970073801212312F800D12320880081232E141
:051BA70080031233BAB7
:0F2AAF00021B98021B9A021B9F021BA4021BA969
:101BAC00900029E090007BF0E566900058F0E56825
:101BBC00900063F0E569900064F0E56A900075F0C0
:101BCC00E56590007DF0E56790007EF0E56490009F
:101BDC0081F0E563900082F090002AE090013BF0E8
:101BEC0090002BE090013CF090002CE090013DF037
:101BFC00900041E0900091F0900042E0900092F053
:101C0C00900043E0900093F0900044E0900094F03A
:101C1C00900045E0900095F0900046E0900096F022
:101C2C00900047E0900097F0900048E0900098F00A
:101C3C00900033E090009AF0900034E090009BF01C
:101C4C00900035E090009CF0900036E090009DF004
:101C5C007400900083F07441900126F0744290015E
:101C6C0027F07436900128F07430900129F074201C
:101C7C0090012AF0744190012BF0743790012CF0F4
:101C8C00743690012DF0743190012EF07445900152
:101C9C002FF07420900130F07436900131F07453B1
:101CAC00900132F07470900133F07464900134F050
:101CBC00900455E0900495F0743A90074FF074FD41
:101CCC00900750F01200C9900004E4F0A3F09000CB
:101CDC00067475F0A37430F09000087475F0A3745A
:101CEC0030F0855859D2CA754C00D29C741B9000A8
:101CFC0023F0E556C394065005E551B55203021E78
:101D0C0009C207E55175F040A4FFAEF09003231211
:101D1C00001EE030E003D38001C39296E55175F0CC
:101D2C0040A4FFAEF090032412001EE030E003D379
:101D3C008001C39295E55175F040A4FFAEF090037D
:101D4C002512001EE030E003D38001C392A0E551C0
:101D5C0075F040A4FFAEF090032612001EE030E0B8
:101D6C0003D38001C39297E560B40206E551640287
:101D7C0060028002D297E552B40506E55164046016
:101D8C00028004C2A28019E55175F040A4FFAEF0A8
:101D9C0090032712001EE030E003D38001C392A20F
:101DAC00E55175F040A4FFAEF090032812001EE040
:101DBC0030E003D38001C3920CE55175F040A4FFD1
:101DCC00AEF090032912001EE030E003D38001C373
:101DDC00920DE560C394045006E560655160028085
:101DEC0002C20D855152AE29AF2A7405BE00039F65
:101DFC005007E545D3940550028002D290E551B4CA
:101E0C000406E55A640A60028019E55175F040A495
:101E1C00FFAEF090032712001EE030E003D38001E8
:101E2C00C392A2900073E06058E54575F00284FF00
:101E3C007E0090014F12001EE0F55CE54775F00A3C
:101E4C0084FF7E0090024F12001EE0F55DE55C25DC
:101E5C005DD39464400BE55C255DC39464F55C80B4
:101E6C0003755C00E55C75F00284FF7E008F5CEF0F
:101E7C00C394335007EF24CDF55C8003755CFF8071
:101E8C001CE54575F00284FF7E0090014F12001E88
:101E9C00E075F00284FF7E00EF24CDF55CE556D3AF
:101EAC00940550030220C3C207E551D3940150039B
:101EBC00021F99E55175F040A4FFAEF090031F127C
:101ECC00001EE0A829B80007D3952A40021551E559
:101EDC005165527003021F96E55175F040A4FFAE98
:101EEC00F090032312001EE030E003D38001C39274
:101EFC0096E55175F040A4FFAEF090032412001E3D
:101F0C00E030E003D38001C39295E55175F040A415
:101F1C00FFAEF090032512001EE030E003D38001E9
:101F2C00C392A0E55175F040A4FFAEF090032612C9
:101F3C00001EE030E003D38001C39297E55175F0A9
:101F4C0040A4FFAEF090032712001EE030E003D354
:101F5C008001C392A2E55175F040A4FFAEF090034E
:101F6C002812001EE030E003D38001C3920CE5512F
:101F7C0075F040A4FFAEF090032912001EE030E093
:101F8C0003D38001C3920D8551520220C3E556B490
:101F9C00065B9000ADE030E003D38001C3929690D5
:101FAC0000AEE030E003D38001C392959000AFE027
:101FBC0030E003D38001C392A09000B0E030E00386
:101FCC00D38001C392979000B1E030E003D380013D
:101FDC00C392A29000B2E030E003D38001C3920C14
:101FEC009000B3E030E003D38001C3920DE556B40A
:101FFC0007659000A6E030E003D38001C392969071
:10200C0000A7E030E003D38001C392959000A8E0D4
:10201C0030E003D38001C392A09000A9E030E0032C
:10202C00D38001C392979000AAE030E003D38001E3
:10203C00C392A29000ABE030E003D38001C3920CBA
:10204C009000ACE030E003D38001C3920DE55AD38D
:10205C00940A4003755CCDE556B4085B90009FE094
:10206C0030E003D38001C392969000A0E030E003EF
:10207C00D38001C392959000A1E030E003D380019E
:10208C00C392A09000A2E030E003D38001C39297EA
:10209C009000A3E030E003D38001C392A29000A48F
:1020AC00E030E003D38001C3920C9000A5E030E057
:1020BC0003D38001C3920DE595C3955C4004C29394
:1020CC008002D293A207B34005E556B4070375739B
:1020DC00CDE595C395734004C2948002D294E54536
:1020EC0075F00284FF7E0090018112001EE075F0F5
:1020FC000284FF7E00EF24CDF56FE595C3956F50FC
:10210C0006A20CB3B340028004D2928002C292E5C4
:10211C004575F00284FF7E009001B312001EE0753D
:10212C00F00284FF7E00EF24CDF570E595C3957029
:10213C005006A20DB3B340028004D2878002C2873E
:10214C00E543C394064003022772A2EDB350030289
:10215C002772C2EDE54360030222B17E017F00E5E8
:10216C00BE124385E5BD2FFF50010E900000EEF02E
:10217C00A3EFF0900029E0B401177E0F7FFF9000D1
:10218C0000E0FCA3E0FD120003900000EEF0A3EFD2
:10219C00F090007AE0B4025B900000E0FEA3E0FF58
:1021AC0090000AE0FCA3E0FDEDD39FEC9E400F9065
:1021BC000000E0F8A3E090000AC8F0A3C8F090007B
:1021CC0000E0FEA3E0FF90000CE0FCA3E0FDEFD3E9
:1021DC009DEE9C400F900000E0F8A3E090000CC82E
:1021EC00F0A3C8F0900000E0FEA3E0FF74041243DB
:1021FC00778F4490007AE07060900000E0FEA3E0DE
:10220C00FF90000AE0FCA3E0FDEFD39DEE9C400D97
:10221C00120003900000EEF0A3EFF0800790000096
:10222C00E4F0A3F0900000E0FEA3E0FF7410124372
:10223C0085900026E08E048F05FF12436790000006
:10224C00ECF0A3EDF07400D39D74019C4008900059
:10225C0001E0F54480037544FFE54475F00AA4FFE2
:10226C00AEF074198E048F05FF1243678D45ED2572
:10227C0032FFAE3150010E74011243778F45854504
:10228C0032753100EFD39462400375456290007350
:10229C00E064016006900067E06002800575430110
:1022AC00800375BB17E543B4010280030223A17EB2
:1022BC00017F00E5BE124385E5BD2FFF50010E9056
:1022CC000000EEF0A3EFF0900073E0B4017EE53473
:1022DC0045336025AC33AD341DBDFF011C8F028E20
:1022EC00038C068D07903EBB12002EE493FE740106
:1022FC0093FFEFC39AEE9B4002800578331243AFF5
:10230C00AE33AF3474B3BE0025D39F402190000090
:10231C00E0FCA3E0FD0FBF00010E903EBB12002EAF
:10232C00E493FE740193FFEDC39FEC9E4002800585
:10233C00783312003FAE33AF34E56A1243857464D0
:10234C008E048F05FF1243678D478033900067E042
:10235C00602D900000E0FEA3E0FFEFD39400EE941C
:10236C0008400F900067E0B40104C2098002D20952
:10237C00800D900067E0B40104D2098002C209907C
:10238C000073E064026006900067E0600575BB16A0
:10239C008003754302E543B40202800302248F7E5E
:1023AC00017F00E5BE124385E5BD2FFF50010E9065
:1023BC000000EEF0A3EFF0900073E0B4027EE53481
:1023CC0045336025AC33AD341DBDFF011C8F028E2F
:1023DC00038C068D0790402512002EE493FE7401A9
:1023EC0093FFEFC39AEE9B4002800578331243AF04
:1023FC00AE33AF3474B3BE0025D39F4021900000A0
:10240C00E0FCA3E0FD0FBF00010E90402512002E52
:10241C00E493FE740193FFEDC39FEC9E4002800594
:10242C00783312003FAE33AF34E56A1243857464DF
:10243C008E048F05FF1243678D478033900067E051
:10244C00602D900000E0FEA3E0FFEFD39400EE942B
:10245C0008400F900067E0B40104C2098002D20961
:10246C00800D900067E0B40104D2098002C209908B
:10247C000073E07003754700900067E07002C209BA
:10248C0075BB1FE543B403457E017F00E5BE1243D7
:10249C0085E5BD2FFF50010E900000EEF0A3EFF08C
:1024AC00740912438574E68E048F05FF1243678C02
:1024BC00418D42E54A2DFD50010C74018C068D07AF
:1024CC001243778E418F4285424A75BB19E543B45E
:1024DC000402800302265A7E017F00E5BE1243856A
:1024EC00E5BD2FFF50010E900000EEF0A3EFF0744D
:1024FC00041243778F4BE564B4010280030225C4B8
:10250C00756B00756B00E56BD3940740030225B126
:10251C00E56B90004112439DE0D3954B501AE56B4F
:10252C0090004112439DE0F404254BFEE56B9000B6
:10253C003712439DEEF08017E56B90004112439DDE
:10254C00E0C3954BFEE56B90003712439DEEF0E532
:10255C006BC394044009900085E0C3956B503BE538
:10256C006B6029E56B90003712439DFEE0FFEE9007
:10257C00003FE0D39F4013E56B90003712439DE082
:10258C0090003FF0E56B900040F0800E900037E03B
:10259C0090003FF07400900040F0786B740126F6C8
:1025AC004003022512900040E0F4042408F556E59F
:1025BC0056D394054002C290E564D39401402FE5B4
:1025CC004BD3946E4004D2118002C211755605E5AE
:1025DC0064B40205A211B340028003755607E5648A
:1025EC00B40306A211B3B340028003755607E55736
:1025FC006556602BE556B40703755A00E556B405CD
:10260C000DE557D394054006E55164016002800C3A
:10261C0075510690004E7401F0755A00855657E5B9
:10262C0056B40708E5B54480F5B58006E5B5547F8A
:10263C00F5B5E55664066005E556B40808E5B544FD
:10264C0010F5B58006E5B554EFF5B575BB13E5434C
:10265C00B40502800302276E7E017F00E5BE1243A3
:10266C0085E5BD2FFF50010E900000EEF0A3EFF0BA
:10267C0074041243778F46E563B402028003022789
:10268C006B756B00756B00E56BD3940340030227ED
:10269C0022E56B90003312439DE0D39546501AE52A
:1026AC006B90003312439DE0F4042546FEE56B90DD
:1026BC00002D12439DEEF08017E56B900033124312
:1026CC009DE0C39546FEE56B90002D12439DEEF008
:1026DC00E56B6029E56B90002D12439DFEE0FFEE4B
:1026EC00900031E0D39F4013E56B90002D12439D79
:1026FC00E0900031F0E56B900032F0800E90002DF0
:10270C00E0900031F07400900032F0786B74012688
:10271C00F64003022693900083E07043E52A452996
:10272C006036E558C39403500A900032E004C39419
:10273C000340028007900032E004F558E558D3942A
:10274C0002400A900032E004D394025002800790B9
:10275C000032E004F5588007900032E004F558751B
:10276C00BB180543D2ECE55ED39404500302293E1A
:10277C0075CF01C293AE35AF367488D39F74139E58
:10278C004005A2A5B34014AE35AF367488D39F7400
:10279C00139E4005A2A4B340028048783512003F36
:1027AC00AE35AF36EFB4883BEEB41337A2A5B350B9
:1027BC0009900050E0D395515002800405518011CE
:1027CC00A2A5B35008900050E0655160028002D27F
:1027DC0007A2A4B35007E551D3940150028004150D
:1027EC0051C207A2A5B3B35006A2A4B3B340028052
:1027FC0006753600753500E551655270030228C028
:10280C00E55175F040A4FFAEF090032312001EE0DA
:10281C0030E003D38001C39296E55175F040A4FFDC
:10282C00AEF090032412001EE030E003D38001C30D
:10283C009295E55175F040A4FFAEF090032512007F
:10284C001EE030E003D38001C392A0E55175F04047
:10285C00A4FFAEF090032612001EE030E003D380FC
:10286C0001C39297E55175F040A4FFAEF090032799
:10287C0012001EE030E003D38001C392A2E5517533
:10288C00F040A4FFAEF090032812001EE030E003ED
:10289C00D38001C3920CE55175F040A4FFAEF090CB
:1028AC00032912001EE030E003D38001C3920DC255
:1028BC0094855152A20740057573CD80037573FF43
:1028CC00E595C395734004C2948002D294E5457596
:1028DC00F00284FF7E0090018112001EE075F00270
:1028EC0084FF7E00EF24CDF56FE595C3956F500600
:1028FC00A20CB3B340028004D2928002C292E5458E
:10290C0075F00284FF7E009001B312001EE075F09A
:10291C000284FF7E00EF24CDF570E595C3957050D1
:10292C0006A20DB3B340028004D2878002C2870294
:10293C00277CA210B3500DAE25AF2674E8C39F744C
:10294C00039E4002800B75FFA0D210E5B554FBF539
:10295C00B5AE25AF26EFD39420EE944E5003022A49
:10296C00711204D5C28E758D00758B00754C00D21A
:10297C008EC2077572007571007573CD7551067531
:10298C002400752300755400755A00E5B554BFF545
:10299C00B590005AE06004D20F8002C20F90004A3A
:1029AC00E0B40108E5B54420F5B58006E5B554DF83
:1029BC00F5B5900049E0B40104D2A18002C2A1A2F5
:1029CC0009B34004D2918002C29190006CE060186F
:1029DC00123B44A200B34008E5B54408F5B58006A7
:1029EC00E5B554F7F5B58002C20090006FE06018B1
:1029FC00123C99A202B34008E5B54402F5B5800635
:102A0C00E5B554FDF5B58013A20FB34008E5B54408
:102A1C0002F5B58006E5B554FDF5B590000E74FDD4
:102A2C00F0A374E8F0E543B4060375430090002569
:102A3C00E4F0752600752500758D00758B00754CBE
:102A4C0000900024E0C394035008900024E004F0AC
:102A5C0080067403900024F0900024E0B40306E593
:102A6C00B554FEF5B5AE27AF28EFD39410EE9427EE
:102A7C00401CC2CA75CD0075CC00752800752700A6
:102A8C00D2CA754E00752A00752900755500020DC5
:012A9C002910
:103E4B00000001000132016401960196020002128A
:103E5B0002240200020003000340038003C004009D
:103E6B000440048004C0050006000600060006009E
:103E7B00060006000600060000FF013101630195F4
:103E8B0001FF01FF0211022302FF02FF02FF033FAA
:103E9B00037F03BF03FF043F047F04BF04FF05FF41
:103EAB0006FF06FF06FF06FF06FF06FF06FF06FFDF
:103EBB000FAA0FA50F9F0F9A0F940F8D0F870F80CF
:103ECB000F780F710F680F600F570F4E0F450F3B99
:103EDB000F300F250F1A0F0E0F020EF50EE80EDB2B
:103EEB000ECC0EBE0EAE0E9F0E8E0E7D0E6C0E5AAF
:103EFB000E470E340E200E0C0DF70DE20DCB0DB54B
:103F0B000D9D0D850D6D0D540D3A0D200D050CE914
:103F1B000CCE0CB10C940C760C580C3A0C1B0BFB06
:103F2B000BDB0BBB0B9A0B790B570B350B130AF1F6
:103F3B000ACE0AAB0A870A640A400A1C09F809D49C
:103F4B0009B0098C09670943091F08FB08D608B299
:103F5B00088E086A0846082307FF07DC07B907968F
:103F6B0007730751072F070D06EC06CA06AA068929
:103F7B0006690649062A060A05EC05CD05B0059229
:103F8B0005750558053C0520050504EA04CF04B565
:103F9B00049C04820469045104390422040B03F4C5
:103FAB0003DE03C803B2039D038903750361034D4D
:103FBB00033B03280316030402F202E102D102C001
:103FCB0002B002A0029102820273026502570249FB
:103FDB00023C022F02220216020901FD01F201E648
:103FEB0001DB01D001C601BB01B101A7019D019409
:103FFB00018B018201790170016801600158015048
:10400B000148014101390132012B0125011E011823
:10401B000111010B010500FF00FA0FA60FA00F996C
:10402B000F920F8B0F840F7C0F740F6B0F620F5857
:10403B000F4E0F430F380F2C0F1F0F120F050EF7DC
:10404B000EE80ED80EC80EB70EA50E930E800E6C92
:10405B000E580E420E2C0E150DFD0DE40DCB0DB1B1
:10406B000D950D790D5D0D3F0D200D010CE10CC073
:10407B000C9E0C7C0C590C350C100BEA0BC40B9ED4
:10408B000B760B4F0B260AFD0AD40AAA0A800A5597
:10409B000A2A09FF09D409A8097C0950092508F93E
:1040AB0008CD08A10875084A081E07F307C8079D25
:1040BB0007730749072006F706CE06A6067E0657A6
:1040CB000630060A05E405BF059B05770554053246
:1040DB00051004EF04CE04AE048F047104530435B1
:1040EB00041903FD03E203C703AD0394037B0363CE
:1040FB00034B0334031E030802F302DE02CA02B6AB
:10410B0002A30291027F026D025C024C023C022C64
:10411B00021D020E020001F201E401D701CA01BE29
:10412B0001B101A6019A018F0185017A0170016627
:10413B00015D0153014A014101390131012901217D
:10414B0001190112010B010400FD00F700F000EA58
:10415B0000E400DE00D900D300CE00C900C400BFCC
:10416B0000BA00B500B100AD00A800A400A0009CEF
:10417B00009900950091008E008A008700840081D1
:04418B00007E007B37
:102ABE00751A00751900AE19AF1AAC17AD18EDC323
:102ACE009FEC9E401674FF12435775CF01781A740F
:102ADE000126F6500418E436F650DB22900787E400
:102AEE00F0A3F0751000750F00751300751400C279
:102AFE0012D21322C2AF75D900758F0375B7A575A3
:102B0E00B7F190F800E4F0758F0175B7A575B7F1C0
:102B1E00E50890F800F075B7A575B7F190F801E4E7
:102B2E00F075B7A575B7F190079EE090F802F075B5
:102B3E00B7A575B7F19007A2E090F803F075B7A5A9
:102B4E0075B7F190079FE090F804F075B7A575B7CB
:102B5E00F19007A0E090F805F075B7A575B7F19064
:102B6E0007A1E090F806F075B7A575B7F19007A329
:102B7E00E090F807F0758F0075D940D2AF2290071C
:102B8E0089E0B4AB61C2AF75D90075B62275F52276
:102B9E00758F0375B7A575B7F1740090F600F075D3
:102BAE008F01750A00750900AE09AF0A7413BE00D5
:102BBE00279F402475B7A575B7F190078A12001E9E
:102BCE00E0FC90F60012001EECF0780A740126F676
:102BDE00500418E436F650D0758F0075F51175B6A1
:102BEE002075D940D2AF22C2AF75D90075F52275C6
:102BFE000A00750900AE09AF0A7413BE00229F4089
:102C0E001F90F60012001EE493FC90078A12001E1D
:102C1E00ECF0780A740126F6500418E436F650D516
:102C2E0075F51175D940D2AF22900789E0B4AA028A
:102C3E008003022D74C2AF75D90075B62275F522C8
:102C4E00758F0375B7A575B7F1740090EE00F0752A
:102C5E00B7A575B7F1740090F000F075B7A575B70C
:102C6E00F1740090F200F075B7A575B7F17400908D
:102C7E00F400F0758F01750A00750900AE09AF0AF0
:102C8E0074FFC39F74019E402475B7A575B7F1906C
:102C9E00004F12001EE0FC90EE0012001EECF078C9
:102CAE000A740126F6500418E436F650CF750A0061
:102CBE00750900AE09AF0A74FFC39F74019E4024CC
:102CCE0075B7A575B7F190024F12001EE0FC90F09B
:102CDE000012001EECF0780A740126F6500418E477
:102CEE0036F650CF750A00750900AE09AF0A74FFAB
:102CFE00C39F74019E402475B7A575B7F190044F1C
:102D0E0012001EE0FC90F20012001EECF0780A7425
:102D1E000126F6500418E436F650CF750A007509F0
:102D2E0000AE09AF0A74FFC39F74019E402475B7AD
:102D3E00A575B7F190064F12001EE0FC90F400123C
:102D4E00001EECF0780A740126F6500418E436F6EC
:102D5E0050CF758F0075F51175B62075D940D2AF6D
:102D6E00743A90074FF022900789E0B4AA028003CC
:102D7E00022EB2C2AF75D90075B62275F522758FC7
:102D8E000375B7A575B7F1740090E600F075B7A599
:102D9E0075B7F1740090E800F075B7A575B7F174CA
:102DAE000090EA00F075B7A575B7F1740090EC00CD
:102DBE00F0758F01750A00750900AE09AF0A74FF30
:102DCE00C39F74019E402475B7A575B7F190004F4F
:102DDE0012001EE0FC90E60012001EECF0780A7461
:102DEE000126F6500418E436F650CF750A00750920
:102DFE0000AE09AF0A74FFC39F74019E402475B7DD
:102E0E00A575B7F190024F12001EE0FC90E800127B
:102E1E00001EECF0780A740126F6500418E436F61B
:102E2E0050CF750A00750900AE09AF0A74FFC39F33
:102E3E0074019E402475B7A575B7F190044F12002A
:102E4E001EE0FC90EA0012001EECF0780A740126D7
:102E5E00F6500418E436F650CF750A00750900AE28
:102E6E0009AF0A74FFC39F74019E402475B7A57500
:102E7E00B7F190064F12001EE0FC90EC0012001EFF
:102E8E00ECF0780A740126F6500418E436F650CFAA
:102E9E00758F0075F51175B62075D940D2AF743A9D
:102EAE0090074FF022900789E0B4AA028003022F08
:102EBE00F0C2AF75D90075B62275F522758F037500
:102ECE00B7A575B7F1740090DE00F075B7A575B7AC
:102EDE00F1740090E000F075B7A575B7F17400902D
:102EEE00E200F075B7A575B7F1740090E400F075C7
:102EFE008F01750A00750900AE09AF0A74FFC39FF2
:102F0E0074019E402475B7A575B7F190004F12005D
:102F1E001EE0FC90DE0012001EECF0780A74012612
:102F2E00F6500418E436F650CF750A00750900AE57
:102F3E0009AF0A74FFC39F74019E402475B7A5752F
:102F4E00B7F190024F12001EE0FC90E00012001E3E
:102F5E00ECF0780A740126F6500418E436F650CFD9
:102F6E00750A00750900AE09AF0A74FFC39F74019C
:102F7E009E402475B7A575B7F190044F12001EE060
:102F8E00FC90E20012001EECF0780A740126F65056
:102F9E000418E436F650CF750A00750900AE09AF75
:102FAE000A74FFC39F74019E402475B7A575B7F1CF
:102FBE0090064F12001EE0FC90E40012001EECF092
:102FCE00780A740126F6500418E436F650CF758F41
:102FDE000075F51175B62075D940D2AF743A9007C9
:102FEE004FF022900789E0B4AA02800302312EC26C
:102FFE00AF75D90075B62275F522758F0375B7A515
:10300E0075B7F1740090D600F075B7A575B7F17469
:10301E000090D800F075B7A575B7F1740090DA007E
:10302E00F075B7A575B7F1740090DC00F0758F01DF
:10303E00750A00750900AE09AF0A74FFC39F7401CB
:10304E009E402475B7A575B7F190004F12001EE093
:10305E00FC90D60012001EECF0780A740126F65091
:10306E000418E436F650CF750A00750900AE09AFA4
:10307E000A74FFC39F74019E402475B7A575B7F1FE
:10308E0090024F12001EE0FC90D80012001EECF0D1
:10309E00780A740126F6500418E436F650CF750AF5
:1030AE0000750900AE09AF0A74FFC39F74019E40FC
:1030BE002475B7A575B7F190044F12001EE0FC9071
:1030CE00DA0012001EECF0780A740126F65004188D
:1030DE00E436F650CF750A00750900AE09AF0A74D2
:1030EE00FFC39F74019E402475B7A575B7F1900676
:1030FE004F12001EE0FC90DC0012001EECF0780A6D
:10310E00740126F6500418E436F650CF758F00750C
:10311E00F51175B62075D940D2AF743A90074FF0BD
:10312E0022C2AF75D90075F522750A00750900AE79
:10313E0009AF0A74FFC39F74019E401F90EE0012E8
:10314E00001EE493FC90004F12001EECF0780A74FF
:10315E000126F6500418E436F650D4750A007509A7
:10316E0000AE09AF0A74FFC39F74019E401F90F01A
:10317E000012001EE493FC90024F12001EECF07839
:10318E000A740126F6500418E436F650D4750A0077
:10319E00750900AE09AF0A74FFC39F74019E401FEC
:1031AE0090F20012001EE493FC90044F12001EECED
:1031BE00F0780A740126F6500418E436F650D475E9
:1031CE000A00750900AE09AF0A74FFC39F74019E11
:1031DE00401F90F40012001EE493FC90064F120064
:1031EE001EECF0780A740126F6500418E436F650F8
:1031FE00D475F51175D940D2AF22C2AF75D900750D
:10320E00F522750A00750900AE09AF0A74FFC39F57
:10321E0074019E401F90E60012001EE493FC900085
:10322E004F12001EECF0780A740126F6500418E4D2
:10323E0036F650D4750A00750900AE09AF0A74FF50
:10324E00C39F74019E401F90E80012001EE493FC81
:10325E0090024F12001EECF0780A740126F650040C
:10326E0018E436F650D4750A00750900AE09AF0A97
:10327E0074FFC39F74019E401F90EA0012001EE46B
:10328E0093FC90044F12001EECF0780A740126F69F
:10329E00500418E436F650D4750A00750900AE09CC
:1032AE00AF0A74FFC39F74019E401F90EC00120082
:1032BE001EE493FC90064F12001EECF0780A740187
:1032CE0026F6500418E436F650D475F51175D9402B
:1032DE00D2AF22C2AF75D90075F522750A007509F5
:1032EE0000AE09AF0A74FFC39F74019E401F90DEAB
:1032FE000012001EE493FC90004F12001EECF078BA
:10330E000A740126F6500418E436F650D4750A00F5
:10331E00750900AE09AF0A74FFC39F74019E401F6A
:10332E0090E00012001EE493FC90024F12001EEC7F
:10333E00F0780A740126F6500418E436F650D47567
:10334E000A00750900AE09AF0A74FFC39F74019E8F
:10335E00401F90E20012001EE493FC90044F1200F6
:10336E001EECF0780A740126F6500418E436F65076
:10337E00D4750A00750900AE09AF0A74FFC39F74B5
:10338E00019E401F90E40012001EE493FC90064F35
:10339E0012001EECF0780A740126F6500418E4367A
:1033AE00F650D475F51175D940D2AF22C2AF75D98A
:1033BE000075F522750A00750900AE09AF0A74FF93
:1033CE00C39F74019E401F90D60012001EE493FC12
:1033DE0090004F12001EECF0780A740126F650048D
:1033EE0018E436F650D4750A00750900AE09AF0A16
:1033FE0074FFC39F74019E401F90D80012001EE4FC
:10340E0093FC90024F12001EECF0780A740126F61F
:10341E00500418E436F650D4750A00750900AE094A
:10342E00AF0A74FFC39F74019E401F90DA00120012
:10343E001EE493FC90044F12001EECF0780A740107
:10344E0026F6500418E436F650D4750A00750900B5
:10345E00AE09AF0A74FFC39F74019E401F90DC003B
:10346E0012001EE493FC90064F12001EECF0780A38
:10347E00740126F6500418E436F650D475F511751D
:10348E00D940D2AF22E51464046006E59964FF606A
:10349E00028031A2124004D2128027E51460087413
:1034AE00E62514900023F0E513600874F0251390C0
:1034BE000023F0E514B4010280FE751400751300AC
:1034CE00C2128002C212E514903DEEF828287375E0
:1034DE001400E599B4FF03751301E599B4FE037565
:1034EE001302E599B4FD03751303E599B4FC037556
:1034FE001304E599B4FA03751305E599B4FB067543
:10350E0014011204D5E599B4F9067514041204D504
:10351E00E599D394E54007E599C394F040028016EF
:10352E008599157514027E017F00E515C394E61288
:10353E0043858E0D8F0E900787E4F0A3F0E599D3A7
:10354E0094C44007E599C394E640028028859915F6
:10355E0075140374E5C39515F50E750D00AE0DAF1C
:10356E000E903E4B12002EE493F874019390078751
:10357E00C8F0A3C8F0D299023A02900787E0FEA3E2
:10358E00E0FFEFC39400EE94054009EFD394FFEEF5
:10359E0094064013900787E0FEA3E0FF90004F12C1
:1035AE00001EE599F0800385996C90078712000E36
:1035BE00900787E0FEA3E0FFEFB40106EEB407022A
:1035CE00800302381290074FE0B43C0280030238A9
:1035DE0012A20AB35005A20BB34003023705C29CD8
:1035EE0090007BE090078DF0900058E090078EF0F1
:1035FE00900063E090078FF0900064E0900790F0E9
:10360E00900075E0900791F090007DE0900792F0A9
:10361E0090007EE0900793F0900081E0900794F088
:10362E00900082E0900795F090013BE0900796F0B5
:10363E0090013CE0900797F090013DE0900798F0E4
:10364E00900091E0900799F0900092E090079AF028
:10365E00900093E090079BF0900094E090079CF010
:10366E00900095E090079DF0900096E090079EF0F8
:10367E00900097E090079FF0900098E09007A0F0E0
:10368E0090009AE09007A1F090009BE09007A2F0C6
:10369E0090009CE09007A3F090009DE09007A4F0AE
:1036AE007400900083F01200C974AB900789F01279
:0A36BE002B8C74AA900789F0E558E0
:063DEE000234DD023588FD
:1036C800903E0FF82828738012122C37800D122D87
:0B36D800758008122EB38003122FF142
:0F3E0F000236CF0236D10236D60236DB0236E05B
:1036E300900789E4F090013BE0700C90013CE0709E
:1036F3000690013DE060028004C20A8002D20A0201
:103703003807C29C900079E090078AF090005FE050
:1037130090078BF0900060E090078CF090007BE0C6
:1037230090078DF0900058E090078EF0900063E0D2
:1037330090078FF0900064E0900790F0900075E0A0
:10374300900791F090007DE0900792F090007EE06A
:10375300900793F0900081E0900794F0900082E04E
:10376300900795F090013BE0900796F090013CE0C4
:10377300900797F090013DE0900798F0900091E05A
:10378300900799F0900092E090079AF0900093E0F0
:1037930090079BF0900094E090079CF0900095E0D8
:1037A30090079DF0900096E090079EF0900097E0C0
:1037B30090079FF0900098E09007A0F090009AE0A7
:1037C3009007A1F090009BE09007A2F090009CE08E
:1037D3009007A3F090009DE09007A4F07400900080
:1037E30083F074AB900789F0122B8C74AA9007892D
:1037F300F0122C37122D75122EB3122FF1D29C75A5
:1038030099FB80FED29C7514007513007599FB0219
:103813003A02900787E0FEA3E0FFEF4E700685991A
:1038230010750F00900787E0FEA3E0FF74016F4E51
:10383300701BAC0FAD10AA0DAB0EED2BFBEC3AFADF
:103843008A068B0790004F12001EE599F0900787B8
:1038530012000E900787E0FEA3E0FF74026F4E7024
:103863000C1200C9851599751400751300023A02EC
:10387300900787E0FEA3E0FF90004F12001EE5993A
:10388300F090078712000E900787E0FEA3E0FFACDD
:103893000DAD0E8F028E038C068D07903E831200B2
:1038A3002EE493F9740193FEEAD39EEB99400985C4
:1038B3001599751400751300023A02900787E0FE0C
:1038C300A3E0FF90004F12001EE599F090078712C6
:1038D300000E900787E0FEA3E0FFEFB40006EEB40E
:1038E30001028003023A0290001CE0D394C7400B0C
:1038F30090001CE0C394C8F516801A90001CE0D316
:103903009463400B90001CE0C39464F5168006900A
:10391300001CE0F516E51675F002A4FFAEF08F6B00
:10392300EF90004F12439DEFFCE0FDEC900052122C
:10393300439DEDFCE0FDEC2DB5160280030239F446
:103943000FEF90004F12439DE56BFFE0FCEF9000FB
:103953005312439DECFFE0FCEFC39CB516028003BA
:103963000239F4E56B90005112439DE56BFFE0FCD7
:10397300EF90005412439DECFFE0FCEF2CB5167161
:10398300E56B90005512439DE0C3951690079EF09A
:10399300E56B90005612439DE0C3951690079FF088
:1039A300E56B90005912439DE0C395169007A0F074
:1039B300E56B90005A12439DE0C395169007A1F062
:1039C300E56B90005B12439DE0C395169007A2F050
:1039D300E56B90005C12439DE0C395169007A3F03E
:1039E300122B027599F9751864751700122ABE8097
:0F39F300FE7599FF751864751700122ABE80FEC5
:093DF4000238150238730238BED2
:103A020022E513903DFDF8282873023B4390078777
:103A1200E0FEA3E0FF90001212001EE0F59990076D
:103A22008712000E900787E0FEA3E0FF74116F4E2D
:103A32007003751300023B43856299023B43900772
:103A420087E0FEA3E0FF90004F12001EE0F599EF21
:103A5200B40107EEB4070375130090078712000E36
:073A6200023B43900788E0DE
:0F3DFD00023A0C023A0F023A3A023A40023A6591
:103A6900903E1EF8282873852499023B38852A99A7
:103A7900023B38854499023B38854799023B388592
:103A89005199023B38856099023B38855699023B2A
:103A990038855899023B38756E0090006AE07006C7
:103AA900900069E060028016A2A44006E56E440415
:103AB900F56EA2A54006E56E4402F56E801A9000E7
:103AC9004AE0B40106E56E4410F56E900049E0B491
:103AD9000106E56E4420F56EA207B34006E56E4483
:103AE90001F56EA209B34006E56E4408F56E856ED0
:103AF90099803CA213B340077599FAC2138017A2A3
:103B09000EB3400575990F800B900023E0F599904D
:103B19000023E4F0C20E80178542998012854B99E3
:0F3B2900800D85469980087599FC8003751300FF
:103E1E00023A70023A76023A7C023A82023A8802FA
:103E2E003A8E023A94023A9A023AA0023AFC023BC5
:0D3E3E0021023B26023B2B023B30023B35AC
:0B3B380090078712000E800312004867
:033E0C00023B4036
:103B43002290006CE0B4010385241190006CE0B472
:103B53000203852A1190006CE0B40303854411909D
:103B6300006CE0B4040385471190006CE0B40503D6
:103B730085511190006CE0B4060385561190006CDA
:103B8300E0B4070385581190006DE0FE90006EE0ED
:103B9300C39E5003023C1A90006CE0D39404402C63
:103BA30090006DE0D39511500990006EE0C395111C
:103BB30050028002D20090006DE0D395115009901D
:103BC300006EE0C395115002C200804990006CE082
:103BD300B4041890006EE0C395115002D200900017
:103BE3006DE0D395114002C200802A90006DE0C3BE
:103BF3009511500990006EE0D3951150028002D2C6
:103C03000090006DE0D39511500990006EE0C395CC
:103C1300115002C200807E90006CE0D39404402CCB
:103C230090006DE0C39511400990006EE0D39511AB
:103C330040028002C20090006DE0C39511400990DC
:103C4300006EE0D395114002D200804990006CE0F1
:103C5300B4041890006DE0C395115002C2009000A7
:103C63006EE0D395114002D200802A90006DE0C32C
:103C73009511400990006EE0D395114002D2009057
:103C8300006DE0D39511400990006EE0C39511409B
:103C9300028002C2002290006FE0B4010385241168
:103CA30090006FE0B40203852A1190006FE0B40323
:103CB3000385441190006FE0B4040385471190001D
:103CC3006FE0B4050385511190006FE0B4060385DE
:103CD300561190006FE0B40703855811900070E00F
:103CE300FE900071E0C39E5003023D6F90006FE0B1
:103CF300D39404402C900070E0D3951150099000A8
:103D030071E0C3951150028002D202900070E0D39B
:103D130095115009900071E0C395115002C20280C1
:103D23004990006FE0B40418900071E0C3951150FE
:103D330002D202900070E0D395114002C202802AA1
:103D4300900070E0C395115009900071E0D3951174
:103D530050028002D202900070E0D3951150099076
:103D63000071E0C395115002C202807E90006FE0A3
:103D7300D39404402C900070E0C395114009900047
:103D830071E0D3951140028002C202900070E0C33B
:103D930095114009900071E0D395114002D2028041
:103DA3004990006FE0B40418900070E0C39511507F
:103DB30002C202900071E0D395114002D202802A20
:103DC300900070E0C395114009900071E0D3951104
:103DD3004002D202900070E0D39511400990007127
:0B3DE300E0C3951140028002C20222E2
:09439D002582F5825002058322FD
:10002E00EF2F500205832582F582E5833E2EF58360
:01003E00229F
:08000300C3EF9DFFEE9CFE22FD
:08003F000806B60002180622B3
:0D000E00A3E004F07006124393E004F0221A
:0843AF000816B6FF02181622E1
:0E437700048007C3CE13CECF13CFD5E0F622BD
:10418F00BC000FBE0008ED8FF084FFADF022E4FEFF
:10419F00FF22BE000DEF60FE54F0606F20E70302B8
:1041AF004245EAC0E0EBC0E078017A0075F001EE1D
:1041BF0020E710EF25E0FFEE33FE0AC5F023C5F030
:1041CF0030E7F0EA5407F9096A7A007B00600108CA
:1041DF00C3EC9E40167004ED9F4010ED9FFDEC9ECA
:1041EF00FCE5F0CA4ACA03F5F08005E5F003F5F0E7
:1041FF00C3EE13FEEF13FFD9D77908CACBCAD8D0B5
:10420F00EAFEEBFFD0E0FBD0E0FA22EC8FF084FC6B
:10421F00ED54F045F0C48FF084FEEDC454F045F03A
:10422F00C48FF084FDEEC4FE54F02DFFEE540F3C0E
:10423F00FEADF07C0022790078008FF0EC7E082034
:10424F00E70DC3CD33CD33C933C9C833C8DEF084CE
:10425F0049F9E5F08FF0BE00E6FD7C00E9FFE8FECE
:01426F00222C
:0E438500F88FF0A4FFE5F0CE88F0A42EFE2203
:10435700600D782B024361007830D8FED5E0F82253
:10436700EEC0E07E0012418FEFFDEEFCD0E0FE22B2
:03000B00024306A7
:03001B000243217C
:03002B0002433C51
:030000000243A612
:0943A60075817475D000020860F5
:0B001E00E5822FF582E5833EF583228A
:0A4393000582D582021583158222EF
:10430600C0E0C0F0C083C082C0D075D0001208558E
:10431600D0D0D082D083D0F0D0E032C0E0C0F0C0A0
:1043260083C082C0D075D000120858D0D0D082D0B9
:1043360083D0F0D0E032C0E0C0F0C083C082C0D0ED
:1043460075D00012085BD0D0D082D083D0F0D0E0F8
:014356003234
:00000001FF
